:040000006F00700518
:1000040000000000000000000406000006060000D6
:100014000000000054080000000000000000000080
:100024005408000054080000000000000000000014
:100034005408000000000000540800000000000004
:10004400540800005408000054080000540800003C
:10005400540800005408000054080000540800002C
:10006400540800005408000054080000540800001C
:10007400540800005408000054080000540800000C
:1000840054080000540800005408000054080000FC
:1000940054080000540800005408000054080000EC
:1000A40054080000540800005408000054080000DC
:1000B400A80500005408000054080000540800007B
:1000C40054080000540800005408000054080000BC
:1000D40054080000540800005408000054080000AC
:1000E400540800005408000054080000540800009C
:1000F400540800005408000054080000540800008C
:1001040054080000540800000000000054080000D7
:10011400540800000000000000000000000000007F
:1001240000000000000000000000000000000000CB
:0C013400000000000000000000000000BF
:10014000397101436EC619A0397141536AC866CA34
:1001500062CC5ECE19A0397101535AD056D252D416
:100160004ED64AD826DA22DC06DE3301614082828E
:1001700041114AC026C222C406C68282B24D410144
:10018000024D924C224CB24B4101024B924A224A00
:10019000B2494101024992442244B2404101828065
:1001A0003D432A876373C3029377F700BDEFADE544
:1001B000937606FF3D8ABA960CC34CC30CC74CC756
:1001C0004107E36BD7FE11E28280B306C3408A0683
:1001D0009702000096966780A6002307B700A30643
:1001E000B7002306B700A305B7002305B700A30493
:1001F000B7002304B700A303B7002303B700A3028B
:10020000B7002302B700A301B7002301B700A30082
:10021000B7002300B700828093F5F50F9396850011
:10022000D58D93960501D58D61B7939627009702DA
:10023000000096968682E78086FA9680C1171D8F09
:100240003E96E374C3F8A5B7EFF29FF23971130637
:10025000000281454808A9378545114502C402C6F8
:1002600002C8EF00706A854513050020EF00D069D1
:100270003165EF00F058371501409307700C2C00E2
:1002800013050580372401407C8402C8EF00F01478
:1002900013050440A12585473ECC3ECEB7070E008E
:1002A0003ED04C089547130504402304F10202CACE
:1002B00002D2EF004065854513050440EF00006B56
:1002C000854513050440EF0060698545130504402A
:1002D000EF00A07B814513050440EF0080791305F2
:1002E0000440EF00C069930404402685EF00C06914
:1002F0006DFD1305044037240140EF00606993044D
:1003000004402685EF0060696DFD1306C00281453B
:100310004808793585450545EF00305DB704024052
:1003200013858400EF00807C9307C4443ECA938702
:1003300001843ECC95473ED0930700083ED49307F6
:1003400000103ED6930700403ED8930700023EDAE5
:100350004C088D67138584003EDC02CE02D202DE9B
:10036000EF00F002138584008545EF00D0051305EA
:1003700004409D4605468145EF0020641305044076
:100380009D4609468545152D130504409D460D469D
:1003900089452525130504409D4611469945312D73
:1003A0009D461546130504409D45012D85451305C1
:1003B0000440C52B2161F9BBEFF29FDB411185455C
:1003C0004145EF0070548D44414989674C00371511
:1003D00001407C824AC626C4EF003000896537158B
:1003E0000140EF00300C8545214537140140EF00F6
:1003F000B051930700204C00130504C07C824AC60C
:1004000026C4EF00807D130504C093050020EF0093
:10041000700985451145EF00304FE177938707104C
:100420004C00130504807C824AC626C4EF00E07AA3
:10043000A1651305048093850510EF00B00685457E
:100440002145EF00704C8567938707804C001305AA
:1004500004C07C824AC626C4EF0020788565130557
:1004600004C093850580EF00F00385452145EF002A
:10047000B04991474C00130504C07C824AC626C48B
:10048000EF00A075130504C09145EF00B00185454C
:100490002145EF007047A1477C824C00914713052E
:1004A00004C03EC626C4EF004073130504C0A14536
:1004B000EF00407F85452145EF0010459307000C74
:1004C0004C00130504C07C824AC626C4EF00E070CD
:1004D0009305000C130504C0EF00007D41015DB9D8
:1004E000EFF21FC9D13D192085336DB1EFF25FC81E
:1004F000011185450545EF001043856793877738DF
:100500003ECA4C089D47370500403ECC231E0100E3
:10051000EF0030450546854537050040EF00504D5A
:100520009307C0027C868D475C87680085473EC87C
:10053000EF00D027854537050040EF00F049056101
:1005400091B9B7170140938707C01307000419C179
:1005500098CB8280D8CB828003D801849387018492
:10056000B623DA239D67938707530953330EF802A6
:10057000B71802009388F8FD33086802469833489C
:100580000E03231005013385F602B3866602B30716
:10059000F702C69633076702B346D5024697B3C73C
:1005A000E70296A11EA28280854537050040EF0034
:1005B000504539C593859181938681819C219822EC
:1005C00013869181850705071377F70F93F7F70FC8
:1005D0009CA198A2A54563F7E50023800600854607
:1005E000A38DD1801307700C6377F70005472300B4
:1005F0000600238DE180854537050040EF00F0417E
:100600007300203001A0B707EFBE37E700E0938703
:1006100007083CC701A0EFF21FB441110545EF00E8
:1006200090187922EF00504E716513050520EF00F8
:10063000B04FB707002083A5070837250000130532
:10064000454BEF00B0594521AA8537250000130519
:10065000454CEF00B05869350545E53523150100D7
:100660002316010023170100054A13840184B72AC9
:10067000000083C7B1816314FA00A38D018083C792
:10068000A181E318FAFE1306E1006C001305A10036
:10069000238D0180D135896537150140FD2B133637
:1006A00015008965371501401125B71401409305E0
:1006B0000020138504C0D5231336150093050020B0
:1006C000138504C0E5231E247A20348730862C85C8
:1006D00013854A4DEF00905069BFEFF27FA93714A0
:1006E00002401C403707FF08411193E717001CC068
:1006F0005C40F98F5CC01C403707F7FE6D17F98F1F
:100700001CC01C403707FCFF7D17F98F1CC05C40E4
:10071000370701FF7D17F98F5CC0B7079F001CC426
:10072000C92502C402C6B727024023A007001C4007
:100730004167B7160240D98F1CC037060200056713
:100740009C42F18F3EC6A24785073EC4B24781E76F
:10075000A247E397E7FEB71702409C431397E700D1
:100760006350070485473EC632478547631CF7023E
:10077000B7170240D843B7160240D8C3D843D8C3EE
:10078000D843D8C3D843719BD8C3D8431367170045
:10079000D8C31147DC42B18BE39EE7FE4101DDBACD
:1007A00002C6D9B7372702401C43F19B1CC3FDB7D3
:1007B000B7160240DC42370700201146B18B130701
:1007C0000708638FC70221466381C70495EB9C42EB
:1007D000918B9DC7B7470F00938707241CC3B7179A
:1007E0000240DC43918393F6F700B707002093871C
:1007F0000700B69794231C43B3D7D7001CC382804D
:10080000B7177A0093870720D1BFDC42D4424166F4
:10081000C983BD8BF18E890745466393C700C947DD
:1008200081EEB746024083A60680C18A89CEB716FC
:100830007A009386062021A8B7160240D442139668
:10084000E600E35606FEB7163D0093860690B38792
:10085000D70269B701A0970100209381A102174137
:1008600000201301217A172500001305E5D397F521
:10087000FF1F938525791386818163FAC500832242
:10088000050023A0550011059105E3EAC5FE138577
:100890008181938501856377B500232005001105CB
:1008A000E36DB5FEFD42739002BC8D4273904280B1
:1008B000930280087390023097F2FFFF9382C27414
:1008C00093E2320073905230EFF03FE19702000064
:1008D0009382A2D47390123473002030B727014062
:1008E000938707406310F502EFF29F888545130553
:1008F0000020EF003005814513050020EF00900433
:100900006FF05F8982805C413707F1E01307F7EFF2
:10091000944D7D8F9C41D58FD44DD58FD441A20667
:10092000D58FD98F5CC11C4537F7F1FF1307D77FEF
:10093000D4457D8F9C49D58F94458606D58FD98F18
:100940001CC55C55370710FF7D177D8FDC29FD170F
:1009500093F7F70FD207D98F5CD582801C4589C5E4
:1009600093E717001CC58280F99BEDBF1C4589C524
:1009700093E707101CC5828093F7F7EFE5BF1C458E
:1009800093E787001CC5828008450D810589828018
:100990001C4593E747001CC58280084509810589ED
:1009A00082801C4591C537075000D98F1CC58280B5
:1009B0003707B0FF7D17F98FD5BFA54763F7B70499
:1009C0008D47138765FF3307F7020328C5009D474E
:1009D000B397E70093C7F7FFB3F70701B396E600B5
:1009E000DD8E54C5994763E3C70495477D163306EA
:1009F000F6025859FD47B397C70093C7F7FFF98F21
:100A00003396C5005D8E50D982800D473387E5024D
:100A1000032805019D47B397E70093C7F7FFB3F796
:100A20000701B396E600DD8E14C96DBFB14763E2DE
:100A3000C702954765163306F6021859FD47B39766
:100A4000C70093C7F7FFF98F3396C5005D8E10D9A5
:100A5000828095474D163306F6025855FD47B397E9
:100A6000C70093C7F7FFF98FB395C500DD8D4CD54F
:100A700082805C4191C537070004D98F5CC18280B8
:100A8000370700FC7D17F98FD5BFB7066745B72735
:100A90000240938636123797EFCDD4C31307B79A27
:100AA000D8C3D4D398C7D85B9386470313162700BF
:100AB000E34B06FED85713670720D8D7DC5B370710
:100AC0000020D98F9CC2372702405C5B9396270099
:100AD000E3DD06FE3C4989C593E707043CC98280F3
:100AE00093F7F7FBE5BF03A5018282801C414167B4
:100AF0007917F98F1CC12320050023220500232428
:100B00000500B707024023260500138787006317F7
:100B1000E500D8431367F700D8C382801387C70165
:100B20006316E500D8431367070FFDB71387070364
:100B30006318E500D8438566938606F0558FE9BFB4
:100B4000138747046315E500D843BD66C5BF138707
:100B500087056316E500D843B7060F00C5B71387AE
:100B6000C7066316E500D843B706F000C1BF138778
:100B700007086316E500D843B706000FC1B713870F
:100B80004709E31CE5F8D843B70600F045BF1C4110
:100B900061773D0794517D8F9C45D58F9449D58FC2
:100BA000D449D58F944DD58FD44DD58FD451D58F71
:100BB0009455D58FD98F1CC1DC455CC19C411CC5A7
:100BC000DC415CC582801C4189C593E717001CC1CC
:100BD000828041677917F98FDDBF9C4513F70701C4
:100BE00013F8F70001C7D8413368E8008E2113F7E6
:100BF000F50F39C318418146854E3D4F930F800252
:100C000093028004214E3396DE00B3F8C5006311D1
:100C100016039398260033131F011343F3FF337712
:100C2000E300B318180133E7E800639FF70550C9E4
:100C30008506E39AC6FD18C11307F00F6375B70464
:100C400054412146854E3D4F930F8002930280040C
:100C5000414EB398CE0033F715016392E8021317A3
:100C6000260001173313EF001343F3FFB376D300CD
:100C70003317E800D98E639DF701232A1501050675
:100C8000E319C6FD54C18280E39457FA10C94DB7E9
:100C9000E39757FE23281501DDB748456D8D3335A1
:100CA000A00082800CC982804CC9828019C20CC904
:100CB00082804CC98280370700C0B377E500639516
:100CC000E708370701405C439356B501584F9D8AAA
:100CD0009DE6F99BB70600FFFD16758F89C993162F
:100CE0000501C182D58FB706FF01758D498FB70603
:100CF0000007D58FB7060140DCC2D8CE82800546FA
:100D00006396C600F59BB70680FFF9B70946639660
:100D1000C600ED9BB706E8FFC1B70D466396C60057
:100D2000DD9BB706FCFF4DBF11466397C60093F7E6
:100D3000F7F3B706C0FF4DB71546E391C6FA93F730
:100D4000F7CFB706E0FF49BF370700406391E702DE
:100D5000B7070140D84F4205B367A70089E513459F
:100D6000F5FFB377E500370701405CCF8280A9E348
:100D700037080140B7073000032648001317050164
:100D8000B376F50041836396F602B70600F9FD16C7
:100D9000B377D60003264800F18E2322D80091C5F0
:100DA000558112053315A700C98F370701405CC371
:100DB00082809317B50063D007029357050193F61D
:100DC000F7008D47B397D70093C7F7FFF18FB706AA
:100DD0000007D58FE9B7935755019207B317F7006E
:100DE000E5B7EFF2EFB837F4FF1F03274472370679
:100DF000003E4111931797019346F7FFF18F0607C5
:100E000037063E00718FD98F370600011397960081
:100E1000718FD98FBD824167F98E02C202C402C6AA
:100E2000D58F23A2F182035784728545239EE180EA
:100E3000032704721305D00323A4E182032744701F
:100E400023A0E182035704732396E182752C832744
:100E5000447037073A101307077093F7F7F063846D
:100E6000E710636BF70037073210130707706380D2
:100E7000E70841016FF00FB237073B101307077007
:100E8000638BE70837073D1013070770E393E7FE0E
:100E9000854521650D3537140140E17793048004C1
:100EA0004C00130504807C8226C6053B856793872A
:100EB00087334C00130504C07C8226C6393B91471A
:100EC0007C824C0093078002130504C03EC6313378
:100ED000F9774C00371501407C8226C6FD398D47D5
:100EE0007C8226C64C0013050440C53959B7E1770A
:100EF0003715014093C707C0130480044C00130545
:100F000005C07C8222C6D13989677C8222C64C000A
:100F100037150140D9BF85452165713B3714014024
:100F2000E177930480044C00130504807C8226C67C
:100F30006D31930700214C00130504C07C8226C646
:100F4000693991477C824C0093078002130504C0E5
:100F50003EC66131F9774C00371501407C8226C6C8
:100F6000AD398947B5BFB7140140E1779387077062
:100F7000130480044C00138504807C8222C6B1399E
:100F8000930790E34C00138504C07C8222C6B131E4
:100F900091477C824C0093078002138504C03EC6B3
:100FA0002D39F9779DB723A8A182828003A70183F9
:100FB000854714216310F7021C31639CE7023C2132
:100FC000960793E707F837E700E093F7F70F3697B0
:100FD0002300F740054793D756003317D7005441F5
:100FE00089CE938707048A07B7E600E0B69798C3CF
:100FF0008280EDF33C219607F9B793870706E5B7A2
:10100000B7160240DC423747FF7F7D17F98F5D8DB1
:10101000C8C28280371702405C439146B18B638C13
:10102000D706A146638ED706BDE71C43918BA5C7A3
:10103000B7470F00938707241CC1371602405C4254
:1010400037070020130707019183BD8BBA979423BC
:101050001C41B3D7D7005CC15442A1829D8ABA9685
:101060009422B3D6D70014C55442AD829D8A3697D8
:101070001423B3D6D70054C55842634C07005C42D2
:10108000B98313F7370093874180BA979C23B3D76E
:10109000F6021CC98280B7177A009387072069BFC0
:1010A0005C435843C166C983BD8B758F8907C546AC
:1010B0006393D700C94701EF3747024003270780F2
:1010C000418B09CF37177A001307072021A837175C
:1010D000024058439316E700E3D606FE37173D005B
:1010E00013070790B387E70281BF99C537170240FE
:1010F0005C4B5D8D48CB8280B7170240D84B1345BF
:10110000F5FF798DC8CB828099C5371702401C4FF7
:101110005D8D08CF8280B7170240984F1345F5FFC9
:10112000798D88CF828099C5371702405C4F5D8DDD
:1011300048CF8280B7170240D84F1345F5FF798D0D
:10114000C8CF828099C5371702405C475D8D48C77C
:101150008280B7170240D8471345F5FF798DC8C77D
:1011600082801E2137370140130707C0C207C183A1
:101170006300E50237070040630CE50013070740F2
:101180006308E50037170040130707806316E50082
:10119000FA2193F7F7F8D98F9A2593F7F7CFC2077B
:1011A000C183D98F371700401EA1130707809C41C8
:1011B0006310E5025CD5DE211EB5B7370140938789
:1011C00007C06314F500BC251EB985475EA982805F
:1011D000C207C1835EB5C5B71E2189C593E7170055
:1011E0001EA18280C207C183F99BC207C183CDBF04
:1011F0005E2501C6DD8D4EA5828093C5F5FFFD8D70
:10120000DDBF1E294A25ED8F4205418189C76D8DBD
:101210003335A00082800145828093C5F5FFC20569
:10122000C1810EA98280EFE2BFF41629F577FD1780
:10123000F58FF621DA257971D58F1EA95625FD7710
:101240009387379FF58FD6212A842EC6D58F962572
:10125000D58FB625D58F5EA55E29C207C18393F7CA
:10126000F7CFD98F5EA968087533B74701409387D8
:101270000780B245631AF404A25756246547B38722
:10128000E702C206C186984163D2060406075224CB
:101290004206B3D7E702130740064186B3D6E702FA
:1012A000B3F7E7029206635506028E07938727037A
:1012B000B3D7E70213F77700B367D700C207C1833C
:1012C0001EA445616FE01FED925745BF0A07C1B7E5
:1012D000920793872703B3D7E702BD8BD58FF9BF5A
:1012E00091C55E250967D98F5EA582805A25F97759
:1012F000FD17F98FD5BF93F5F51F4EA182800A2106
:101300006D8D3335A0008280B707002083A70708C2
:101310000967130707F4B3D7E702C207C183239B0A
:10132000F182239AF1828280EFE29FE42A841165A0
:10133000011185451105C93B930700207C823715B3
:1013400001408D473EC44C00E147130505803EC671
:10135000EFF0BF8822C837440140B70708000C08E7
:10136000130504803ECC02CA231E01006D3D854555
:1013700013050480B53705616FE0DFE1EFE2BFDD03
:10138000B7440140AE8932890144938404806345A7
:1013900024014A856FE07FDF9305000426858537A9
:1013A00065DDB38789008385070026850504C205AE
:1013B000C1819137E9BF138781801C4393860185E2
:1013C0003E95636BD500B75600209386068063E593
:1013D000A60008C33E858280FD57EDBF39713EDA15
:1013E0002ED232D436D63AD842DC46DE9387C1803C
:1013F00022CC804326CA06CEAA8409C41C4C99E399
:101400002285F9200C4454102686228536C6A5264E
:10141000F2406244D24421618280411122C406C656
:101420002A844EA572A5232005002322050023242B
:1014300005002322050623280500232A0500232C66
:101440000500214681451305C505EFE07FD59717B7
:101450000000938767985CD0971700009387879A5E
:101460001CD4971700009387679E5CD497170000E1
:101470009387C7A000D01CD8B2402244410182808B
:1014800097150000938505D4A9A2411126C2130621
:1014900080069384F5FFB384C4024AC02E8922C417
:1014A00006C693854407592A2A8401CD23200500C6
:1014B00023222501310508C4138684068145EFE007
:1014C0003FCE2285B24022449244024941018280AB
:1014D0001C4DADE3411106C622C497070000938757
:1014E00067FA1CD5938701819C4323240504232696
:1014F0000504232805046314F50085471CCD2A84C0
:101500001D2848C02285052808C422852D2048C4EE
:10151000484001469145113708440546A545F53D2B
:1015200048440946C945D53D85471CCCB2402244B4
:1015300041018280828041119387018126C28443C8
:101540004AC006C69C4C22C42A8999E3268549379D
:10155000938484048044DC40FD1763D607009C40DC
:10156000B9CF8440C5BF0317C40039E7C1778507E9
:101570002322040623200400232204002324040041
:101580005CC423280400232A0400232C04002146E1
:1015900081451305C405EFE0BFC0232A0402232CB4
:1015A000040223240404232604042285B240224496
:1015B00092440249410182801304840671BF91451F
:1015C0004A85E13588C051FDB1472320F900014427
:1015D000E9BF797122D44AD052CC56CA5AC85EC6E5
:1015E00006D626D24ECE2A8AAE8A13048504014935
:1015F000054BFD5B09ECB25022544A8592540259C6
:10160000F249624AD24A424BB24B4561828004445D
:1016100083294400FD1963D409000040E1BFDE24A2
:10162000637BFB008397E40063877701A68552857F
:10163000829A3369A90093848406E9BF011126CAFE
:1016400093843500F19806CE22CC4AC84EC6A10438
:10165000B14763F3F404B14463E2B4042A89EF00B0
:10166000304F9387818398433A8439E09387C183CD
:101670009C4391E781454A850D2F23AEA182A68523
:101680004A852527FD5963193507B1472320F900FD
:101690004A85EF00104C29A0E3D004FCB1471CC1DF
:1016A0000145F2406244D2444249B2490561828018
:1016B0001C40858F63CF0702AD4663F6F6001CC061
:1016C0003E9404C031A05C406313870223ACF182D6
:1016D0004A85EF0010481305B40093074400619950
:1016E0003307F5405DDF3A94898F1CC05DBF5CC352
:1016F000C5B72287404095BF130435007198E302B7
:1017000085FCB305A4404A854D25E31C35FBB5BFD8
:101710001C46FD171CC663D90700184E63C5E700B9
:10172000A9476393F500A1AF1C422E8513871700CC
:1017300018C28CA38280011122CC26CA4AC84EC688
:1017400052C406CE2A89AE893284B304D6007D5AAB
:1017500063149400014501A80C204E864A854D3F34
:101760000504E31745FFF2406244D2444249B249BE
:10177000224A05618280357122CD26CB4AC94EC7E7
:1017800006CF52C556C35AC1DEDEE2DCE6DAAA89CC
:10179000AE843289368401C51C4D91E3153B971701
:1017A00000009387A7D86398F40C83A44900DE2433
:1017B000A18BE5C79C48F5C393070002A304F1027F
:1017C0009307000302D22305F10222C6930B5002B5
:1017D000971A0000938A8AD9054C294B4A841C2009
:1017E00099C3639E770DB30C2441638D0C00E6868C
:1017F0004A86A6854E858137FD576301F51E9256B0
:10180000E69636D21C20638B071CFD571309140083
:1018100002C802CE3ECA02CCA309010482D4834589
:10182000090015465685EF00303113041900C247F0
:1018300049E913F7070109C713070002A309E104E7
:1018400013F7870009C71307B002A309E104834611
:1018500009001307A002638EE606F2474A84814618
:101860002546182093051400130707FD6376E60A42
:10187000ADCA3ECEBDA097170000938727CD6395D4
:10188000F40083A4890025B797170000938707C841
:10189000E39FF4F083A4C90019BFA6854E85F12506
:1018A00001DD7D55FA406A44DA444A49BA492A4A78
:1018B0009A4A0A4BF65B665CD65C0D618280050431
:1018C00039BF330555413315AC00C98F3EC8228955
:1018D000B9B7324793064700184336C66347070235
:1018E0003ACE18209307E002631DF70418309307DF
:1018F000A002631BF702B2470904138747009C4309
:101900003AC663C107023ECA2DA83307E04093E7F9
:1019100027003ACE3EC8F1B7B387670385462E84C9
:10192000BA9781B7FD57C5B7050402CA81468147FA
:101930002546182093051400130707FD6376E60675
:10194000F9F20C200D46171500001305A5C2EF0093
:10195000B01E11CD971700009387C7C11D8D930747
:101960000004B397A700424505045D8D2AC80C20EA
:10197000194617150000130525C013091400230488
:10198000B102EF00701B35C197E7FFFF93878767B0
:1019900095E74247B2471377071009CF91073EC634
:1019A0009257D2973ED21DBDB387670385462E84DA
:1019B000BA9741B79D07E19BA107D5B77800970675
:1019C0000000938686D726860C084E859700000077
:1019D000E7000000FD572A8AE314F5FCDE2493F7A4
:1019E0000704E39007EC125575BD780097060000D8
:1019F0009386A6D426860C084E85012AE1BF79710C
:101A000056CA9C49BA8A984522D426D24ECE52CC88
:101A100006D64AD05AC85EC6AA892E84B284368AAF
:101A200063D3E700BA879CC00347340419C3850712
:101A30009CC01C4093F7070281C79C4089079CC04B
:101A40000329040013796900631A0900130B940138
:101A5000FD5B5C449840998F634CF9041C408346BD
:101A6000340493F70702B336D000A5EB1306340411
:101A7000D2854E85829AFD576303F5041C401146BA
:101A80009840998B544481446397C700B384E640DF
:101A900063D3040081441C4418486354F700998FB1
:101AA000BE94014969047D5B63982405014509A83A
:101AB00085465A86D2854E85829A631E75017D556C
:101AC000B250225492540259F249624AD24A424BCD
:101AD000B24B456182800509ADBF3307D4001306C0
:101AE0000003A301C7040347540493871600A29779
:101AF0008906A381E7049DBF85462286D2854E854F
:101B0000829AE30E65FB050945B7797122D426D286
:101B10004AD04ECE06D652CC56CA5AC8B689942D53
:101B2000930790063289AA842E8413863504638D28
:101B3000F60263E2D706930780056385F61863ED26
:101B4000D700638D062093073004638EF60A930A4C
:101B500024042301D404C9A0930730066385F60A40
:101B600093074006E395F6FE1C40084393F60708EA
:101B700093054500C5C61C410CC363D80700130775
:101B8000D002B307F040A301E40497160000938647
:101B9000269F294765A8930700076381F61663E52A
:101BA000D7029307E0066388F6189307F006E390E0
:101BB000F6FA0C401C4313F8050813854700630729
:101BC000080608C39C4385A893075007E383F6FEE5
:101BD000930780076388F61293073007E399F6F6B8
:101BE0001C43D04181459386470014C383AA070054
:101BF0005685992701C53305554148C05C401CC82E
:101C0000A301040461A81C43930A2404938647009B
:101C10009C4314C32301F4048547D5B793F6070406
:101C20001C410CC3B9DAC207C18781BF93F5050413
:101C300008C3C9D99E231307F0066386E60E9716DC
:101C400000009386E6932947A30104044C400CC48A
:101C500063C5050008406D9908C099E3B28A89CD33
:101C6000B28AB3F5E702FD1AB6958C212380BA003B
:101C7000B3D5E70263FFE70AA147631EF7001C40E4
:101C8000858B91CB58401C4863C7E700930700033E
:101C9000A38FFAFEFD1A3306564110C84E87CA8636
:101CA0007000A2852685A13B7D5A631D450B7D559D
:101CB000B250225492540259F249624AD24A424BDB
:101CC00045618280A382D504971600009386468BD7
:101CD0000C40084313F805081C411105630D080268
:101CE00008C313F7150001C793E505020CC041476F
:101CF000A1FF0C4093F5F5FD0CC0B9B79C4193E7EB
:101D000007029CC193078007A302F4049716000002
:101D10009386468875BF13F8050408C3E30308FCDF
:101D2000C207C1837DBF9716000093866685214751
:101D300021BFAE873DB794411C43CC4913F8060838
:101D4000138547006306080008C39C438CC339A071
:101D500008C393F606049C43F5DA8EA323280400F7
:101D6000B28A2DBF14485686CA8526858299E3001B
:101D700045F51C40898B8DE7B2474844E35AF5F29C
:101D80003E853DB785465686CA8526858299E300FD
:101D900065F3050A5C443247998FE345FAFEE9BFD3
:101DA000014A930A94017D5BF5B7411122C42A844C
:101DB0002E8523A6018406C6EFF0EFDFFD576317DB
:101DC000F5009387C1849C4391C31CC0B240224458
:101DD00041018280411122C42E848395E50006C60C
:101DE000212D634905007C48AA977CC8B240224453
:101DF000410182805E247D777D17F98F5EA4FDB757
:101E0000DE25011122CC26CA4AC84EC606CE93F75B
:101E10000710AA842E843289B68991C78395E5007C
:101E20008946014609215E247D777D17F98F5EA4DE
:101E30008315E4006244F240CE864A86B2494249A4
:101E40002685D2440561DDA8411122C42E848395E4
:101E5000E50006C6C92EFD575A24631AF500FD7722
:101E6000FD17F98F5EA4B24022444101828085674C
:101E7000D98F5EA468C8C5BF8395E500F5A201119E
:101E800022CC26CA4AC806CE4EC6AA842E893284DF
:101E900009C51C4D99E3EFF0AFE397070000938766
:101EA000E7686317F406C0401C4C1CC45E24A18B79
:101EB000C1C31C48B5CF1C4808409379F90F13796A
:101EC000F90F1D8D5C486346F500A2852685CD2C53
:101ED00025E51C440505FD171CC41C40138717008D
:101EE00018C0238037015C486388A7005E24858B77
:101EF00081CBA9476316F900A2852685D1240DED73
:101F0000F24062444A85D2444249B2490561828026
:101F100097070000938787636314F400804469B7D0
:101F2000970700009387875EE310F4F8C044ADBFC5
:101F3000A28526851D2841D17D59D9B7411122C4DA
:101F40002A842E85B285368623A6018406C6EFF044
:101F5000EFC2FD576317F5009387C1849C4391C37B
:101F60001CC0B24022444101828041119387C1804C
:101F700026C2844322C44AC006C62A892E8491C43C
:101F80009C4C81E72685EFF0AFD49707000093873C
:101F9000E759631BF402C0400317C40093170701FD
:101FA000C18393F68700ADEA93F6070195EEA54746
:101FB0002320F900136707045AA47D55B240224438
:101FC0009244024941018280970700009387075895
:101FD0006314F4008044C9B7970700009387075340
:101FE000E31CF4FAC0444DBF918B9DC34C5889C982
:101FF000930744046384F5004A85A92E232A04022A
:102000005E242322040093F7B7FD5EA41C481CC085
:102010005E2493E787005EA41C4899EB5E241307B7
:10202000002093F707286385E700A2854A85AD2C39
:102030005E2413F717001DC35C4823240400B30774
:10204000F0401CCC1C480145B5FB8317C40013F7B6
:1020500007082DD793E707045EA485B7898B01474E
:1020600091E3584818C4F9BF411122C42A842E852F
:1020700023A6018406C60121FD576317F500938747
:10208000C1849C4391C31CC0B24022444101828060
:10209000DE25011122CC26CA06CE4AC84EC613F749
:1020A0008700AA842E8479EBD841634DE000B841C3
:1020B000634AE0000145F2406244D2444249B249D9
:1020C0000561828058547DD703A904009396370197
:1020D00023A0040063DB060670485E24918B99C739
:1020E0005C401D8E5C5899C33C401D8E5C540C5066
:1020F000814626858297FD575A24631DF50094403A
:10210000F54763E8D706B70740208507B3D7D70060
:10211000858BA5C31C48232204001CC093173701DC
:1021200063D80700FD576314F5009C4091E368C82D
:102130004C5823A02401BDDD930744046384F500BB
:102140002685092C232A0402B5B70C500146854682
:1021500026850297FD572A86E311F5F89C40B5DFE6
:1021600075476385E70059476393E70423A024017B
:1021700091B7136707045AA47D5535BF83A905019C
:10218000E38A09F203A905008D8B23A035013309E9
:102190003941014791E3D84918C4E35D20F11C544B
:1021A0000C50CA864E86268582976347A0005E241F
:1021B00093E707045EA4C9B7AA993309A940F1BF00
:1021C0009C49A5C3011122CC06CE2A8419C51C4DF9
:1021D00089E72EC6EFF0CFAFB2459707000093878F
:1021E000E734639BF5004C408397C50095C7228573
:1021F0006244F240056169BD970700009387073587
:102200006394F5000C44CDB797070000938707301F
:10221000E39CF5FC4C44C9BFF240624401450561B2
:10222000828001458280411122C42A842E85B28594
:10223000368623A6018406C68D24FD576317F50054
:102240009387C1849C4391C31CC0B2402244410186
:1022500082801971A6DAAE848395E500A2DC86DE61
:10226000328463DB0500DE2423A0060093F7070811
:102270009DE39307004015A0300836C66522B2469C
:10228000E34305FE7247BD67F98F7977BA9793B735
:1022900017009CC2F9BF930700041CC0F650665497
:1022A000D654014509618280DE25011122CC06CE7B
:1022B00026CA4AC8898B2E8489CF930774041CC010
:1022C0001CC885475CC8F2406244D244424905615B
:1022D000828074003000AA84AD3FA2452A892685F9
:1022E000EFF0CFB519E98317C40013F7072061FF9A
:1022F000F19B93E727005EA4C9B797F7FFFF938789
:1023000067189CD45E2408C008C893E707085EA439
:10231000A2475CC8B24799CB8315E4002685052AFD
:1023200011C55E24F19B93E717005EA45E24336918
:10233000F9002316240141BF93F5F50F2A96631483
:10234000C500014582801C21E38EB7FE0505C5BF8F
:1023500082808280CDC183A7C5FF411122C406C6F9
:1023600026C21384C5FF63D307003E94AA84CD37E9
:10237000938781839C4399EB2322040023AC8182C1
:102380002244B240268592444101E1B7637EF400C5
:1023900014403307D4006396E7009843DC43369734
:1023A00018C05CC0E1BFBA87D84319C3E37DE4FE1F
:1023B00094433386D700631F86001040B29694C3BF
:1023C0003386D700E31EC7FA10435843B29694C32E
:1023D000D8C37DB76375C400B1479CC055B71040E2
:1023E000B306C4006316D70014435843B29614C012
:1023F00058C0C0C371B78280411122C42A842E857F
:10240000B285368623A6018406C67128FD57631758
:10241000F5009387C1849C4391C31CC0B240224401
:1024200041018280411122C42A842E85B28523A6CF
:10243000018406C6B920FD576317F5009387C18450
:102440009C4391C31CC0B24022444101828041118F
:1024500022C42A842E8523A6018406C60D28FD5792
:102460006317F5009387C1849C4391C31CC0B2409D
:102470002244410182809307800523A6F1847D5583
:1024800082809307800523A6F1847D55828093077F
:10249000800523A6F184014582809307800523A649
:1024A000F1847D5582809307800523A6F1847D55B4
:1024B0008280000053797374656D436C6B3A2564B8
:1024C0000D0A00004368697049443A253038780D98
:1024D0000A0000000D0A54656D70313A25640D0A3A
:1024E00054656D70323A25640D0A54656D70333A47
:1024F00025640D0A4453473A25640D0A4348473A78
:1025000025640D0A0000000000000000000000002B
:1025100000000000000000000000000000000000BB
:1025200000000000000000000000000000000000AB
:10253000000000000000000000000000000000009B
:10254000000000000000000000000000000000008B
:10255000000000000000000000000000000000007B
:102560000000000000000000232D302B20000000A0
:10257000686C4C0065666745464700003031323371
:10258000343536373839414243444546000000006F
:1025900030313233343536373839616263646566D9
:0425A0000000000037
:1025A40000000000000000000102030406070809FF
:1025B40000000000010203040102030406070809E5
:1025C4000000000028250000482500000825000020
:1025D40000000000000000000000000000000000F7
:1025E40000000000000000000000000000000000E7
:1025F40000000000000000000000000000000000D7
:1026040000000000000000000000000000000000C6
:1026140000000000000000000000000000000000B6
:1026240000127A0002040608D000002020000020D6
:0826340020000020000000005E
:00000001FF
